 gpt

 Timestamp is 4fb04cc5 (Mon May 14 12:07:33 2012)

 Preferred load address is 10000000

 Start         Length     Name                   Class
 0001:00000000 00000004H .CRT$XCA                CODE
 0001:00000004 00000004H .CRT$XCZ                CODE
 0001:00000008 00000004H .CRT$XIA                CODE
 0001:0000000c 00000004H .CRT$XIZ                CODE
 0001:00000010 00000004H .CRT$XPA                CODE
 0001:00000014 00000004H .CRT$XPZ                CODE
 0001:00000018 00000004H .CRT$XTA                CODE
 0001:0000001c 00000004H .CRT$XTZ                CODE
 0001:00000020 00000028H .rdata                  CODE
 0001:00000048 00000020H .rdata$debug            CODE
 0001:00000068 00000fd0H .text                   CODE
 0001:00001038 00000000H .xdata                  CODE
 0001:00001038 0000003cH .idata$2                CODE
 0001:00001074 00000014H .idata$3                CODE
 0001:00001088 00000094H .idata$4                CODE
 0001:0000111c 0000004cH .idata$6                CODE
 0001:00001170 000000ffH .edata                  CODE
 0002:00000000 00000094H .idata$5                DATA
 0002:00000094 00000008H .data                   DATA
 0002:0000009c 00000014H .bss                    DATA
 0003:00000000 00000150H .pdata                  DATA

  Address         Publics by Value              Rva+Base       Lib:Object

 0000:00000000       ___safe_se_handler_table   00000000     <absolute>
 0000:00000000       ___safe_se_handler_count   00000000     <absolute>
 0001:00000000       __xc_a                     10001000     corelib0:crt0init.obj
 0001:00000004       __xc_z                     10001004     corelib0:crt0init.obj
 0001:00000008       __xi_a                     10001008     corelib0:crt0init.obj
 0001:0000000c       __xi_z                     1000100c     corelib0:crt0init.obj
 0001:00000010       __xp_a                     10001010     corelib0:crt0init.obj
 0001:00000014       __xp_z                     10001014     corelib0:crt0init.obj
 0001:00000018       __xt_a                     10001018     corelib0:crt0init.obj
 0001:0000001c       __xt_z                     1000101c     corelib0:crt0init.obj
 0001:0000003c       ??_C@_1M@EENNDIOJ@?$AAI?$AAn?$AAd?$AAe?$AAx?$AA?$AA@ 1000103c     gpt_mx25_topaz_v1:gptpdd.obj
 0001:00000068       BSPGptGetClockSource       10001068 f   bspgpt.obj
 0001:00000090       BSPGptCalculateCompareVal  10001090 f   bspgpt.obj
 0001:0000012c       BSPGptChangeClockSource    1000112c f   bspgpt.obj
 0001:00000138       BSPGptShowClockSource      10001138 f   bspgpt.obj
 0001:0000013c       BSPGptSetClockGatingMode   1000113c f   bspgpt.obj
 0001:000001b8       BSPGptGetBaseAddress       100011b8 f   bspgpt.obj
 0001:00000210       BSPGptGetIRQ               10001210 f   bspgpt.obj
 0001:00000258       GPT_Init                   10001258 f   gpt_common_topaz_v1:gptmdd.obj
 0001:00000268       GPT_Deinit                 10001268 f   gpt_common_topaz_v1:gptmdd.obj
 0001:0000027c       GPT_Open                   1000127c f   gpt_common_topaz_v1:gptmdd.obj
 0001:000002b8       GPT_Close                  100012b8 f   gpt_common_topaz_v1:gptmdd.obj
 0001:000002e4       GPT_PowerDown              100012e4 f   gpt_common_topaz_v1:gptmdd.obj
 0001:0000030c       GPT_PowerUp                1000130c f   gpt_common_topaz_v1:gptmdd.obj
 0001:00000348       GPT_Read                   10001348 f   gpt_common_topaz_v1:gptmdd.obj
 0001:00000350       GPT_Write                  10001350 f   gpt_common_topaz_v1:gptmdd.obj
 0001:00000358       GPT_Seek                   10001358 f   gpt_common_topaz_v1:gptmdd.obj
 0001:00000360       GPT_IOControl              10001360 f   gpt_common_topaz_v1:gptmdd.obj
 0001:000004ec       DllEntry                   100014ec f   gpt_common_topaz_v1:gptmdd.obj
 0001:00000504       DisableThreadLibraryCalls  10001504 f   coredll:COREDLL.dll
 0001:00000514       DDKClockGetFreq            10001514 f   cspddk:CSPDDK.dll
 0001:00000524       DDKClockSetGatingMode      10001524 f   cspddk:CSPDDK.dll
 0001:00000534       _DllEntryCRTStartup        10001534 f   corelib0:pegdentry.obj
 0001:00000678       _cexit                     10001678 f   corelib0:cexit.obj
 0001:00000694       _initterm                  10001694 f   corelib0:crt0dat.obj
 0001:000006c8       _cinit                     100016c8 f   corelib0:crt0dat.obj
 0001:000006fc       __security_init_cookie     100016fc f   corelib0:seccinit.obj
 0001:00000758       __utod                     10001758 f   corelib1:COREDLL.dll
 0001:00000768       __muld                     10001768 f   corelib1:COREDLL.dll
 0001:00000778       __divd                     10001778 f   corelib1:COREDLL.dll
 0001:00000788       __dtou                     10001788 f   corelib1:COREDLL.dll
 0001:00000798       free                       10001798 f   corelib1:COREDLL.dll
 0001:000007a8       __security_gen_cookie2     100017a8 f   corelib1:COREDLL.dll
 0001:000007b8       GptTimerCreateEvent        100017b8 f   gpt_mx25_topaz_v1:gptpdd.obj
 0001:00000808       GptTimerReleaseEvent       10001808 f   gpt_mx25_topaz_v1:gptpdd.obj
 0001:0000083c       GptEnableTimer             1000183c f   gpt_mx25_topaz_v1:gptpdd.obj
 0001:00000880       GptDisableTimer            10001880 f   gpt_mx25_topaz_v1:gptpdd.obj
 0001:000008c0       GptEnableTimerInterrupt    100018c0 f   gpt_mx25_topaz_v1:gptpdd.obj
 0001:000008f0       GptDisableTimerInterrupt   100018f0 f   gpt_mx25_topaz_v1:gptpdd.obj
 0001:0000091c       GptShowClkSrc              1000191c f   gpt_mx25_topaz_v1:gptpdd.obj
 0001:00000944       GptClearInterruptStatus    10001944 f   gpt_mx25_topaz_v1:gptpdd.obj
 0001:0000097c       GptRegInit                 1000197c f   gpt_mx25_topaz_v1:gptpdd.obj
 0001:00000a14       GptRegChangeClkSrc         10001a14 f   gpt_mx25_topaz_v1:gptpdd.obj
 0001:00000a60       GptResetTimer              10001a60 f   gpt_mx25_topaz_v1:gptpdd.obj
 0001:00000aa4       GptGetTimerCount           10001aa4 f   gpt_mx25_topaz_v1:gptpdd.obj
 0001:00000ab8       GptUpdateTimerPeriod       10001ab8 f   gpt_mx25_topaz_v1:gptpdd.obj
 0001:00000b10       GptSetTimerMode            10001b10 f   gpt_mx25_topaz_v1:gptpdd.obj
 0001:00000b64       GptRelease                 10001b64 f   gpt_mx25_topaz_v1:gptpdd.obj
 0001:00000c6c       GptChangeClkSrc            10001c6c f   gpt_mx25_topaz_v1:gptpdd.obj
 0001:00000d0c       GptInitialize              10001d0c f   gpt_mx25_topaz_v1:gptpdd.obj
 0001:00000ea8       DeleteCriticalSection      10001ea8 f   coredll:COREDLL.dll
 0001:00000eb8       InterlockedExchange        10001eb8 f   coredll:COREDLL.dll
 0001:00000ec8       TerminateProcess           10001ec8 f   coredll:COREDLL.dll
 0001:00000ed8       EnterCriticalSection       10001ed8 f   coredll:COREDLL.dll
 0001:00000ee8       InitializeCriticalSection  10001ee8 f   coredll:COREDLL.dll
 0001:00000ef8       LeaveCriticalSection       10001ef8 f   coredll:COREDLL.dll
 0001:00000f08       EventModify                10001f08 f   coredll:COREDLL.dll
 0001:00000f18       GetLastError               10001f18 f   coredll:COREDLL.dll
 0001:00000f28       CreateEventW               10001f28 f   coredll:COREDLL.dll
 0001:00000f38       CloseHandle                10001f38 f   coredll:COREDLL.dll
 0001:00000f48       InterruptDone              10001f48 f   coredll:COREDLL.dll
 0001:00000f58       WaitForSingleObject        10001f58 f   coredll:COREDLL.dll
 0001:00000f68       LocalFree                  10001f68 f   coredll:COREDLL.dll
 0001:00000f78       InterruptDisable           10001f78 f   coredll:COREDLL.dll
 0001:00000f88       KernelIoControl            10001f88 f   coredll:COREDLL.dll
 0001:00000f98       CeSetThreadPriority        10001f98 f   coredll:COREDLL.dll
 0001:00000fa8       CreateThread               10001fa8 f   coredll:COREDLL.dll
 0001:00000fb8       InterruptInitialize        10001fb8 f   coredll:COREDLL.dll
 0001:00000fc8       RegCloseKey                10001fc8 f   coredll:COREDLL.dll
 0001:00000fd8       RegQueryValueExW           10001fd8 f   coredll:COREDLL.dll
 0001:00000fe8       OpenDeviceKey              10001fe8 f   coredll:COREDLL.dll
 0001:00000ff8       LocalAlloc                 10001ff8 f   coredll:COREDLL.dll
 0001:00001008       MmUnmapIoSpace             10002008 f   ceddk:CEDDK.dll
 0001:00001018       MmMapIoSpace               10002018 f   ceddk:CEDDK.dll
 0001:00001028       strcmp                     10002028 f   corelib1:COREDLL.dll
 0001:00001038       __IMPORT_DESCRIPTOR_COREDLL 10002038     coredll:COREDLL.dll
 0001:0000104c       __IMPORT_DESCRIPTOR_CSPDDK 1000204c     cspddk:CSPDDK.dll
 0001:00001060       __IMPORT_DESCRIPTOR_CEDDK  10002060     ceddk:CEDDK.dll
 0001:00001074       __NULL_IMPORT_DESCRIPTOR   10002074     coredll:COREDLL.dll
 0002:00000000       __imp_MmMapIoSpace         10003000     ceddk:CEDDK.dll
 0002:00000004       __imp_MmUnmapIoSpace       10003004     ceddk:CEDDK.dll
 0002:00000008       \177CEDDK_NULL_THUNK_DATA  10003008     ceddk:CEDDK.dll
 0002:0000000c       __imp_DisableThreadLibraryCalls 1000300c     coredll:COREDLL.dll
 0002:00000010       __imp___utod               10003010     corelib1:COREDLL.dll
 0002:00000014       __imp___muld               10003014     corelib1:COREDLL.dll
 0002:00000018       __imp___divd               10003018     corelib1:COREDLL.dll
 0002:0000001c       __imp___dtou               1000301c     corelib1:COREDLL.dll
 0002:00000020       __imp_free                 10003020     corelib1:COREDLL.dll
 0002:00000024       __imp___security_gen_cookie2 10003024     corelib1:COREDLL.dll
 0002:00000028       __imp_DeleteCriticalSection 10003028     coredll:COREDLL.dll
 0002:0000002c       __imp_InterlockedExchange  1000302c     coredll:COREDLL.dll
 0002:00000030       __imp_TerminateProcess     10003030     coredll:COREDLL.dll
 0002:00000034       __imp_EnterCriticalSection 10003034     coredll:COREDLL.dll
 0002:00000038       __imp_InitializeCriticalSection 10003038     coredll:COREDLL.dll
 0002:0000003c       __imp_LeaveCriticalSection 1000303c     coredll:COREDLL.dll
 0002:00000040       __imp_EventModify          10003040     coredll:COREDLL.dll
 0002:00000044       __imp_GetLastError         10003044     coredll:COREDLL.dll
 0002:00000048       __imp_CreateEventW         10003048     coredll:COREDLL.dll
 0002:0000004c       __imp_CloseHandle          1000304c     coredll:COREDLL.dll
 0002:00000050       __imp_InterruptDone        10003050     coredll:COREDLL.dll
 0002:00000054       __imp_WaitForSingleObject  10003054     coredll:COREDLL.dll
 0002:00000058       __imp_LocalFree            10003058     coredll:COREDLL.dll
 0002:0000005c       __imp_InterruptDisable     1000305c     coredll:COREDLL.dll
 0002:00000060       __imp_KernelIoControl      10003060     coredll:COREDLL.dll
 0002:00000064       __imp_CeSetThreadPriority  10003064     coredll:COREDLL.dll
 0002:00000068       __imp_CreateThread         10003068     coredll:COREDLL.dll
 0002:0000006c       __imp_InterruptInitialize  1000306c     coredll:COREDLL.dll
 0002:00000070       __imp_RegCloseKey          10003070     coredll:COREDLL.dll
 0002:00000074       __imp_RegQueryValueExW     10003074     coredll:COREDLL.dll
 0002:00000078       __imp_OpenDeviceKey        10003078     coredll:COREDLL.dll
 0002:0000007c       __imp_LocalAlloc           1000307c     coredll:COREDLL.dll
 0002:00000080       __imp_strcmp               10003080     corelib1:COREDLL.dll
 0002:00000084       \177COREDLL_NULL_THUNK_DATA 10003084     coredll:COREDLL.dll
 0002:00000088       __imp_DDKClockGetFreq      10003088     cspddk:CSPDDK.dll
 0002:0000008c       __imp_DDKClockSetGatingMode 1000308c     cspddk:CSPDDK.dll
 0002:00000090       \177CSPDDK_NULL_THUNK_DATA 10003090     cspddk:CSPDDK.dll
 0002:00000094       __security_cookie          10003094     corelib0:seccinit.obj
 0002:00000098       __security_cookie_complement 10003098     corelib0:seccinit.obj
 0002:0000009c       TICKS_PER_S_IPGCLK         1000309c     bspgpt.obj
 0002:000000a0       _exitflag                  100030a0     corelib0:cexit.obj
 0002:000000a4       __onexitend                100030a4     <common>
 0002:000000a8       __onexitbegin              100030a8     <common>
 0002:000000ac       g_pcsExit                  100030ac     <common>

 entry point at        0001:00000534

 Static symbols

 0001:0000057c       doexit                     1000157c f   corelib0:cexit.obj
 0001:00000cac       GptIntrThread              10001cac f   gpt_mx25_topaz_v1:gptpdd.obj
